:10000000000000000000CB298030A100FE30C62097
:100010000130C6207530AB0030301B29A101A1177B
:10002000B900FE30C6203908C628A701B200B301C6
:10003000A01127080319A0150530A6002730AF002E
:1000400010302E200330AF00E8302E20AF01643096
:100050002E20AF010A302E2032083528AE0033089A
:10006000AB003208AA0071212A08AA00A6030319CE
:10007000A011270803193F282602031846282A083A
:10008000031DA011A0194628303EC6280800A01163
:100090002708031D4E28A0150A30A7003D08AD0013
:1000A0003C08AC003B08AB003A08AA00A601B50129
:1000B000B401B3010A30B2003B21A60A2608270288
:1000C000031D57283208031DA011A01D6928270B06
:1000D0006C283208303EC620A70B4E28C729B7002F
:1000E000051185118316051185110510061085105F
:1000F000861083123708A0189B283E30AB00803052
:100100001B213330B600AF201330AB0088301B21E9
:10011000AF2064301A21AF2064301A212230B6009B
:10012000AF2028309A200C309A2006309A20A01454
:1001300037089B282014B600201CA9288511033CF1
:10014000031CAE28AE200730AB00D0301B210314B7
:1001500008002014FE3C0319C4288515201C20101B
:10016000051500000514361E05100614B61E0610EF
:100170008514361F85108614B61F86100511B60E1D
:100180002018AF2832301A213708C729A11B6F2841
:10019000080083169B0083169C011C141A089B0AF6
:1001A000C72983169A001C1555309D00AA309D0062
:1001B0009C149C18D9281C119B0AC7290830B6002A
:1001C0002918AF212308840024082919BE21291DDC
:1001D000C021220884002809841780052208840091
:1001E000AB0CAA0C00082804031C28068000FB2086
:1001F000B60BEE28C72923088400240880062A08A5
:10020000AE002B08AF00AB0164301B212E08AA0002
:100210002F08AB00240880060800AF01AE00FF30B5
:10022000AE07031CAF07031CC7290330AB00DF3048
:100230001B210F29AB01E83EAA00AB09FC30031CCF
:100240002429AA0703182129AA070000AB0F212996
:100250002A182A29AA1C2E2900002E290800013E4E
:10026000A5000A30B200B301B401B5013B21A50BD2
:10027000312932080800BE01BF01C001C10121308F
:10028000B0006229BE0DBF0DC00DC10D32083E0287
:100290003308031C330F3F023408031C340F4002A1
:1002A0003508031C350F4102031C6229C1003208C6
:1002B000BE023308031C330FBF023408031C340F83
:1002C000C0020314AA0DAB0DAC0DAD0DB00B42294D
:1002D0004108B5004008B4003F08B3003E08B20032
:1002E000C729B301B2011030B6002B0DB20DB30D0A
:1002F0002E08B2022F08031C2F0FB3020318872900
:100300002E08B2072F0803182F0FB3070310AA0DEA
:10031000AB0DB60B75292A0808002030B600BE01C7
:10032000BF01C001C10103102A1CA4293208BE0765
:1003300033080318330FBF0734080318340FC007FE
:1003400035080318350FC107C10CC00CBF0CBE0C1B
:10035000AD0CAC0CAB0CAA0CB60B93290800AE018B
:10036000AF01B629AB0CAA0CAE0DAF0DFF3E0318C2
:10037000B2292F08AB002E08AA00C7298004C32980
:10038000FF3A8005C429FF3A84178005C7298313E3
:100390008312031308008301A00107309F00F0308F
:1003A0008316850086018312DF013030DE00D430F1
:1003B000DD00DC015030D900DB018030DA00003094
:1003C000C920C900CB20CA00CB20CB00CB20CC0059
:1003D0005F08AD005E08AC005D08AB005C08AA00D9
:1003E0005A08B2005B08B300B401B5013B212D08E7
:1003F000E3002C08E2002B08E1002A08E000D0010D
:10040000CF01CE01CD013030C920E6002130C92016
:10041000ED000130AF002C300E2104208030A1000F
:100420000E2020306F202A306F2020306F202A309D
:100430006F2020306F2054306F2020306F204130EB
:100440006F2020306F2032306F2020306F204530F9
:100450006F2020306F2049306F2020306F202A30ED
:100460006F2020306F202A306F2020306F208030A6
:10047000A100C0300E2037306F2030306F20633045
:100480006F206D306F202E306F2020306F20413074
:100490006F204C306F2049306F2043306F2049303F
:1004A0006F2020306F202D306F2020306F2056308D
:1004B0006F2045306F2052306F2069306F204330FD
:1004C0006F2069306F200330AF00E8300E21042028
:1004D000851A6B2A6B24051A722A831686138312D7
:1004E0008617762A8316861383128613051BB52A70
:1004F0005830C9079E3003110318013E031DCA0777
:10050000FF3003110318013E031DCB07FF30031119
:100510000318013E031DCC074C081A3C031CAC2AEF
:10052000031DA22A4B082C3C031CAC2A031DA22A43
:100530004A08E53C031CAC2A031DA22A4908AF3C2B
:10054000031CAC2A1A3083120313CC002C30CB00CE
:10055000E530CA00B030C900E6035A30660203181D
:10056000B32A5A30E60064300D21851BEC2AA830EE
:10057000C907613003186230CA0701300318CB077E
:1005800001300318CC071A304C02031CE32A031D68
:10059000D92A31304B02031CE32A031DD92A173014
:1005A0004A02031CE32A031DD92AE9304902031C2D
:1005B000E32A1A3083120313CC003130CB001730FA
:1005C000CA00E830C900E60A66306602031CEA2A5F
:1005D0006530E60064300D21303083169B008312B5
:1005E0006608D120051E072BC0304907D500893089
:1005F00003188A304A07D6004630031847304B07A5
:10060000D7000130031802304C07D800192BC03036
:100610004907D5002830031829304A07D6006B3027
:1006200003186C304B07D7000130031802304C0719
:10063000D80055084D02031D292B56084E02031DF4
:10064000292B57084F02031D292B58085002031964
:10065000682A831203135808D0005708CF005608A1
:10066000CE005508CD005808AD005708AC0056081C
:10067000AB005508AA006308B5006208B400610821
:10068000B3006008B2003B212D08C5002C08C4004F
:100690002B08C3002A08C2004508AD004408AC007E
:1006A0004308AB004208AA00B501B401B3015908E0
:1006B000B2003B212B08C7002A08C6004608AA0042
:1006C0004708AB00AC01AD01B501B401B301590855
:1006D000B2008D212D08BD002C08BC002B08BB00EA
:1006E0002A08BA003A084202C800051E802B4C08AE
:1006F000D4004B08D3004A08D2004908D100952BFA
:10070000C0305507D100DF30D20056080318560F0D
:10071000D2072030D30057080318570FD307FE30F5
:10072000D40058080318580FD4075408AD005308D4
:10073000AC005208AB005108AA00B5010F30B4005C
:100740004230B3004030B2003B212B08E5002A08BC
:10075000E4005408AD005308AC005208AB00510847
:10076000AA0005302F21E7005408AD005308AC0063
:100770005208AB005108AA0004302F21E8005408A9
:10078000AD005308AC005208AB005108AA0003307A
:100790002F21E900D8233F2483169B0183124908A7
:1007A000D1204A08D1204B08D1204C08D120682AFA
:1007B00004208030A1000E204B306F2041306F208C
:1007C0004E306F2041306F204C306F203A306F2018
:1007D00020306F2052306F20660815208030A10035
:1007E000C0300E2046306F2072306F202E306F20C8
:1007F00020306F203A306F20A7016408B2006508EE
:10080000B30018202E306F206708152068081520C7
:100810006908152020306F204D306F2048306F2040
:100820007A306F208030A10094300E2056306F2037
:1008300043306F204F306F2020306F203A306F20D0
:1008400020306F20A7015808BD005708BC0056088B
:10085000BB005508BA0047208030A100D4300E20DC
:1008600046306F2052306F20A7014C08BD004B0866
:10087000BC004A08BB004908BA004720080083169C
:100880000612831206160330AA00AA0B452C00009C
:100890000630A2000430A8000630A3000830A400EF
:1008A0000130A900AA01DF20AA010130DF2046089B
:1008B000AA004708AB000A30DF204808AA0007302A
:1008C000DF200330AA00AA0B632C00008316061257
:1008D00083120612080004208030A1000E2043304D
:1008E0006F2054306F2043306F2053306F206F20C3
:1008F00020306F2041306F2079306F2061306F20C1
:1009000072306F206C306F2061306F206D306F203F
:1009100061306F200330AF00E8300E2104208030BA
:10092000A1000E2054306F204F306F204E306F20CA
:1009300020306F203A306F2085300E206F08152050
:100940002E306F20700815208B300E2048306F201D
:100950007A306F208030A100C0300E2020306F2010
:100960004F306F204B306F2020306F2069306F2068
:100970004C306F2045306F2020306F2053306F2077
:1009800045306F2043306F20851EF42D051BC92C88
:10099000ED0301306D020318CF2C0130ED006430FF
:1009A0000D21851BD42CED0A1A306D02031CDA2CA4
:1009B0001930ED0064300D2101306D02031DE42C6F
:1009C0000230EB009E30EA0002306D02031DEC2C79
:1009D0000230EB00B630EA0003306D02031DF42C48
:1009E0000230EB00CF30EA0004306D02031DFC2C16
:1009F0000230EB00E830EA0005306D02031D042DE3
:100A00000330EB000230EA0006306D02031D0C2DAE
:100A10000330EB001D30EA0007306D02031D142D7A
:100A20000330EB003930EA0008306D02031D1C2D45
:100A30000330EB005630EA0009306D02031D242D0F
:100A40000330EB007530EA000A306D02031D2C2DD7
:100A50000330EB009330EA000B306D02031D342DA0
:100A60000330EB00B430EA000C306D02031D3C2D66
:100A70000330EB00CE30EA000D306D02031D442D33
:100A80000330EB00E830EA000E306D02031D4C2D00
:100A90000430EB000B30EA000F306D02031D542DC3
:100AA0000430EB003030EA0010306D02031D5C2D85
:100AB0000430EB005530EA0011306D02031D642D47
:100AC0000430EB007C30EA0012306D02031D6C2D07
:100AD0000430EB00A430EA0013306D02031D742DC6
:100AE0000430EB00CE30EA0014306D02031D7C2D83
:100AF0000430EB00F930EA0015306D02031D842D3F
:100B00000530EB002630EA0016306D02031D8C2DF7
:100B10000530EB005530EA0017306D02031D942DAF
:100B20000530EB008530EA0018306D02031D9C2D66
:100B30000530EB00B630EA0019306D02031DA42D1C
:100B40000530EB00EA30EA006D086E020319C42C90
:100B50006B08AB006A08AA00AF010A30AE00712131
:100B6000EF006B08AB006A08AA00AF010A30AE00C4
:100B700071213208F00004208030A1000E20543092
:100B80006F204F306F204E306F2020306F203A3072
:100B90006F2085300E206F0815202E306F207008D2
:100BA00015208B300E2048306F207A306F20803037
:100BB000A100C0300E2020306F204F306F204B300E
:100BC0006F2020306F2069306F204C306F2045300F
:100BD0006F2020306F2053306F2045306F2043301E
:100BE0006F206D08EE00C42C04208030A1000E2080
:100BF00043306F2054306F2053306F206F202030EF
:100C00006F2054306F204F306F204E306F205530A2
:100C10006F203A306F2020306F206F0815202E3063
:100C20006F207008152020306F2048306F207A30F8
:100C30006F208030A100C0300E204F306F204C302C
:100C40006F2041306F2052306F2041306F204B3089
:100C50006F2020306F2053306F2045306F2043309D
:100C60006F2069306F204C306F2044306F20693026
:100C70006F20213083169B0083126D08D120033032
:100C8000AF00E8300E210630A2002030A800063068
:100C9000A3004030A4000130A900AA010230DF20E7
:100CA0006D08AA000630DF2004208030A1000E204D
:100CB0004B306F2041306F204E306F2041306F201D
:100CC0004C306F203A306F2020306F2052306F2030
:100CD000660815208030A100C0300E2046306F20FD
:100CE00072306F202E306F2020306F203A306F200E
:100CF000A7016408B2006508B30018202E306F20E9
:100D000067081520680815206908152020306F2015
:100D10004D306F2048306F207A306F208030A10036
:100D200094300E2056306F2043306F204F306F20AC
:100D300020306F203A306F2020306F20A7015808F4
:100D4000BD005708BC005608BB005508BA00472034
:100D50008030A100D4300E2052306F2058306F20E8
:100D600054306F2058306F200030051A01301520A4
:040D70000800B92E90
:02400E00503F21
:00000001FF
